:100000000C9462000C948A000C948A000C948A0070
:100010000C948A000C948A000C948A000C948A0038
:100020000C948A000C948A000C948A000C948A0028
:100030000C948A000C948A000C948A000C948A0018
:100040000C94C4010C948A000C9446020C948A000F
:100050000C948A000C948A000C948A000C948A00F8
:100060000C948A000C948A000000000024002700F1
:100070002A0000000000250028002B0000000000DE
:1000800023002600290004040404040404040202DA
:100090000202020203030303030301020408102007
:1000A0004080010204081020010204081020000012
:1000B0000007000201000003040600000000000029
:1000C00000008F0311241FBECFEFD4E0DEBFCDBFF1
:1000D00011E0A0E0B1E0E2EEFAE002C005900D927E
:1000E000A231B107D9F711E0A2E1B1E001C01D9240
:1000F000A83BB107E1F710E0C4ECD0E004C02297C0
:10010000FE010E946B05C23CD107C9F70E940101A4
:100110000C946F050C9400000F931F93CF93DF9303
:10012000809102010E947501EC01809104010E94FE
:1001300075018C018091120190911301C817D907A4
:1001400039F480911401909115010817190729F1CC
:10015000809102010E947501BC0185EA91E00E9434
:10016000DE0485EA91E060E071E00E940004809185
:1001700004010E947501BC0185EA91E00E94DE0441
:1001800085EA91E00E940804809116019091170180
:1001900001969093170180931601809106016C2FB0
:1001A0000E942801D0931301C093120110931501EE
:1001B00000931401DF91CF911F910F91089585EA6B
:1001C00091E040E855E260E070E00E948302809197
:1001D000020160E00E9408018091020161E00E943A
:1001E00028018091040160E00E94080180910401CF
:1001F00061E00E9428018091060161E00E940801EF
:1002000008950E940C020E94DF000E948C00FDCF26
:10021000282F30E0C90186569F4FFC0194912A5740
:100220003F4FF9018491882391F0E82FF0E0EE0F21
:10023000FF1FE859FF4FA591B491662329F48C91D3
:10024000909589238C9308958C91892B8C93089594
:10025000482F50E0CA0182559F4FFC012491CA01EA
:1002600086569F4FFC0194914A575F4FFA01349193
:100270003323D1F1222331F1233021F48091800006
:100280008F7705C0243031F4809180008F7D80937A
:10029000800018C0213019F484B58F7704C0223053
:1002A00021F484B58F7D84BD0DC0263021F480916A
:1002B000B0008F7705C0273029F48091B0008F7D82
:1002C0008093B000E32FF0E0EE0FFF1FEE58FF4FDA
:1002D000A591B491662329F48C91909589238C93F0
:1002E00008958C91892B8C930895682F70E0CB0131
:1002F00082559F4FFC012491CB0186569F4FFC01F4
:1003000044916A577F4FFB019491992319F420E09F
:1003100030E038C0222331F1233021F48091800075
:100320008F7705C0243031F4809180008F7D8093D9
:10033000800018C0213019F484B58F7704C02230B2
:1003400021F484B58F7D84BD0DC0263021F48091C9
:10035000B0008F7705C0273029F48091B0008F7DE1
:100360008093B000892F90E0880F991F84589F4F89
:10037000FC01A591B4918C9120E030E0842311F030
:1003800021E030E0C90108951F920F920FB60F923D
:1003900011242F933F938F939F93AF93BF9380919B
:1003A0001C0190911D01A0911E01B0911F0130917F
:1003B00020010196A11DB11D232F2D5F2D3720F0A7
:1003C0002D570196A11DB11D2093200180931C0182
:1003D00090931D01A0931E01B0931F0180911801FD
:1003E00090911901A0911A01B0911B010196A11DD4
:1003F000B11D8093180190931901A0931A01B09335
:100400001B01BF91AF919F918F913F912F910F90C1
:100410000FBE0F901F901895789484B5826084BDAC
:1004200084B5816084BD85B5826085BD85B58160F8
:1004300085BDEEE6F0E0808181608083E1E8F0E058
:10044000808182608083808181608083E0E8F0E049
:10045000808181608083E1EBF0E080818460808333
:10046000E0EBF0E0808181608083EAE7F0E080816A
:1004700084608083808182608083808181608083CA
:100480008081806880831092C10008951F920F922E
:100490000FB60F9211242F933F934F935F936F9357
:1004A0007F938F939F93AF93BF93EF93FF9340916D
:1004B000C600E091A101F091A201CF01019660E890
:1004C00070E00E9405059C018091A3019091A40118
:1004D0002817390739F0EF5DFE4F40833093A201B2
:1004E0002093A101FF91EF91BF91AF919F918F91C7
:1004F0007F916F915F914F913F912F910F900FBE20
:100500000F901F9018955F926F927F928F929F929B
:10051000AF92BF92CF92DF92EF92FF920F931F9311
:10052000CF93DF93EC013A014B01413482E4580749
:100530008FE0680780E078070CF07FC060E874E81F
:100540008EE190E0A40193010E943A0521503040D1
:1005500040405040CA01B90122E030E040E050E0A4
:100560000E943A0559016A01A6019501209530952E
:100570004095509594E0220F331F441F551F9A95C4
:10058000D1F760E074E284EF90E00E943A05CA017E
:10059000B9012FEF30E040E050E00E94E604A401F2
:1005A00093010E943A05C90181509F4F1816190600
:1005B0001CF4522E5A9403C055245394521A60E0EE
:1005C00079E08DE390E0A40193010E943A05215067
:1005D000304040405040CA01B90122E030E040E0E4
:1005E00050E00E943A05209530954095509583E063
:1005F000220F331F441F551F8A95D1F760E074E224
:1006000084EF90E00E943A05CA01B9012FEF30E073
:1006100040E050E00E94E604A40193010E943A05E4
:10062000C90181509F4F181619061CF4822F815062
:1006300002C081E0821B851500F5E885F98581E01F
:1006400090E00A8802C0880F991F0A94E2F780831D
:1006500060E079E08DE390E0A40193010E943A0507
:100660002150304040405040CA01B90122E030E002
:1006700040E050E00E943A0504C0E885F985108208
:100680009501EC81FD813083EE81FF812083EA8535
:10069000FB85208141E050E0CA010E8402C0880F32
:1006A000991F0A94E2F7282B2083EA85FB85208195
:1006B000CA010F8402C0880F991F0A94E2F7282B01
:1006C0002083EA85FB858081088802C0440F551F7E
:1006D0000A94E2F7842B8083DF91CF911F910F91D1
:1006E000FF90EF90DF90CF90BF90AF909F908F9052
:1006F0007F906F905F900895FC01A085B18521895E
:100700008C9190E0022E02C0959587950A94E2F7AD
:1007100080FFF6CF0484F585E02D608308958CE09A
:1007200091E09093A6018093A50181E291E09093DE
:10073000A8018093A70185EC90E09093AA01809393
:10074000A90184EC90E09093AC018093AB0180EC24
:1007500090E09093AE018093AD0181EC90E0909396
:10076000B0018093AF0186EC90E09093B20180934A
:10077000B10184E08093B30183E08093B40187E00A
:100780008093B50185E08093B60181E08093B70145
:1007900008950F931F93CF93DF938C01EB0109C052
:1007A0002196D801ED91FC910190F081E02DC801D6
:1007B000099568816623A1F7DF91CF911F910F9171
:1007C0000895EF92FF920F931F93CF93DF938C01C5
:1007D0007B01EA010CC0D7016D917D01D801ED913B
:1007E000FC910190F081E02DC80109952197209797
:1007F00091F7DF91CF911F910F91FF90EF900895A6
:10080000DC01ED91FC910280F381E02D09950895C2
:100810000F931F938C01DC01ED91FC910190F0810D
:10082000E02D6DE00995D801ED91FC910190F081EA
:10083000E02DC8016AE009951F910F9108952F924C
:100840003F924F925F926F927F928F929F92AF9260
:10085000BF92CF92DF92EF92FF920F931F93DF939D
:10086000CF93CDB7DEB7A0970FB6F894DEBF0FBE1B
:10087000CDBF1C016A017B01411551056105710560
:1008800049F4DC01ED91FC910190F081E02D60E3F1
:10089000099554C0882499245401422E5524662475
:1008A000772401E010E00C0F1D1F080D191DC70172
:1008B000B601A30192010E941805F8016083089413
:1008C000811C911CA11CB11CC701B601A30192019E
:1008D0000E941805C901DA016C017D01C114D1041F
:1008E000E104F104F1F681E0E82EF12CEC0EFD1E9E
:1008F000E80CF91C3E010894611C711CD501C4016F
:100900000197A109B1096C01C818D90814C0F601F2
:10091000EE0DFF1D60816A3010F4605D01C0695CFE
:10092000D101ED91FC910190F081E02DC10109957B
:100930000894E108F1086E147F0449F7A0960FB6F9
:10094000F894DEBF0FBECDBFCF91DF911F910F9105
:10095000FF90EF90DF90CF90BF90AF909F908F90DF
:100960007F906F905F904F903F902F900895EF92FF
:10097000FF920F931F93CF93DF93EC017A018B01CA
:1009800077FF0FC0E881F9810190F081E02D6DE2E1
:10099000099510950095F094E094E11CF11C011D5F
:1009A000111DCE01B801A7012AE00E941F04DF91AA
:1009B000CF911F910F91FF90EF900895AB016627A3
:1009C00057FD6095762F0E94B7040895629FD0016D
:1009D000739FF001829FE00DF11D649FE00DF11DFA
:1009E000929FF00D839FF00D749FF00D659FF00DA9
:1009F0009927729FB00DE11DF91F639FB00DE11D96
:100A0000F91FBD01CF011124089597FB092E072678
:100A10000AD077FD04D049D006D000201AF4709592
:100A200061957F4F0895F6F7909581959F4F0895B2
:100A3000A1E21A2EAA1BBB1BFD010DC0AA1FBB1FE2
:100A4000EE1FFF1FA217B307E407F50720F0A21B54
:100A5000B30BE40BF50B661F771F881F991F1A94C1
:100A600069F760957095809590959B01AC01BD01EB
:100A7000CF01089597FB092E05260ED057FD04D00F
:100A8000D7DF0AD0001C38F4509540953095219559
:100A90003F4F4F4F5F4F0895F6F7909580957095B3
:100AA00061957F4F8F4F9F4F0895AA1BBB1B51E14C
:100AB00007C0AA1FBB1FA617B70710F0A61BB70BCE
:100AC000881F991F5A95A9F780959095BC01CD0173
:100AD0000895EE0FFF1F0590F491E02D0994F8940E
:020AE000FFCF46
:100AE20020000B000C000D00000000007C03C90375
:020AF200E1031E
:00000001FF
